:020000040000FA
:06020000A8EF19F0120046
:0602080016EF01F01200E8
:02022A000000D2
:04022C00DACFE4FF42
:10023000E2CFDAFFE9CFE4FFEACFE4FFE6529EA087
:1002400080D0FE0ECF6E0C0ECE6E300E81140001EB
:10025000C46FC851C45D41E0C851300A28E0100A9B
:1002600018E0200A08E0C4B930D0822B000E8323A6
:10027000842385232FD0C4AB06D0822B000E83238A
:100280008423852305D08207000E835B845B855B16
:1002900022D0C4A906D0822B000E83238423852379
:1002A00005D08207000E835B845B855B14D0C4BBE2
:1002B00006D0822B000E83238423852305D082075A
:1002C000000E835B845B855B06D08207000E835B38
:1002D000845B855B00D0C4C0C8F0C5050CE1180E76
:1002E000C16EC651040DF350C26EA40EC06EC28022
:1002F000020EC56F10D0020EC55D04E1C282030E6E
:10030000C56F09D0030EC55D06E1C250020B03E1C3
:10031000040EC56FC290C75101E0C707B22B000E93
:10032000B323D00EB25D070EB35905E3CC2B010EFB
:10033000CD6FB26BB36BC95103E0C90701E1D76B55
:100340009E909EAA33D00001D95110E0AECFC4F0E8
:10035000D9070AE0D851D82BEA6ADA0FE96E000E05
:10036000EA22EF50AD6E01D0AC9A20D0ABA205D0FE
:10037000AECFC4F0AB98AB8819D0ABA406D09EAA80
:1003800003D0AECFC4F0FBD711D09EAA0DD0080E7B
:10039000D75D09E2D751D72BEA6ACF0FE96E000E7D
:1003A000EA22AECFEFFFF1D7140EC96FE552E5CFC9
:1003B000EAFFE5CFE9FFE5CFDAFF1100D9CFE6FF8D
:1003C000E1CFD9FFE652FD0EDBCF14F0FE0EDBCFFE
:1003D00015F0070ED89015321432E804FBE10E0E2A
:1003E0001414DF6EC580C5B0FED79E96A00EDF2424
:1003F000C96E9EA6FED79E96FF0EE76EFD0EDBCF62
:1004000014F0FE0EDBCF15F0E7501416156A1450E9
:10041000C96E9EA6FED79E96C582C5B2FED79E9691
:10042000A10EDF10C96E9EA6FED79E96C5869EA61B
:10043000FED79E96C950DF6EC58AC588C5B8FED75F
:10044000C584C5B4FED7DF5000D0E552E552E7CFF2
:10045000D9FF1200D9CFE6FFE1CFD9FFC580C5B0E3
:10046000FED79E96FD0EDBCF14F0FE0EDBCF15F00F
:10047000070ED89015321432E804FBE10E0E141664
:10048000000E1516A00E1424C96E9EA6FED79E96C9
:10049000FF0EE76EFD0EDBCF14F0FE0EDBCF15F086
:1004A000E7501416156A1450C96E9EA6FED79E9684
:1004B000FC0EDB50C96E9EA6FED79E96C584C5B4C1
:1004C000FED7E552E7CFD9FF1200D9CFE6FFE1CF43
:1004D000D9FFFA0EDB5022E0FD0EDBCF14F0DB2A51
:1004E000FE0EDBCF15F001E3DB2A14C0E6FF15C0DA
:1004F000E6FF64DFE552E552E66EFB0EDBCFE9FF77
:10050000FC0EDBCFEAFFE552E750EF6EFB0EDB2A75
:10051000FC0E01E3DB2AFA0EDB06DBD7E552E7CF60
:10052000D9FF1200D9CFE6FFE1CFD9FFC580C5B012
:10053000FED79E96FD0EDBCF14F0FE0EDBCF15F03E
:10054000070ED89015321432E804FBE10E0E141693
:10055000000E1516A00E1424C96E9EA6FED79E96F8
:10056000FF0EE76EFD0EDBCF14F0FE0EDBCF15F0B5
:10057000E7501416156A1450C96E9EA6FED79E96B3
:10058000FA0EDB5013E0FB0EDBCFE9FFFC0EDBCFF6
:10059000EAFFEF50C96E9EA6FED79E96FB0EDB2AA1
:1005A000FC0E01E3DB2AFA0EDB06EAD7C584C5B4EC
:1005B000FED7E552E7CFD9FF1200D9CFE6FFE1CF52
:1005C000D9FF0001CE350AE3CE5102E0960ECA6F84
:1005D000809A8490BA6A8282CE6B14D0809A84808A
:1005E000FE0EDB40E8403F0BBB6EFE0EDB50030B04
:1005F000100DF3500C09BA6ECE0502E0960ECA6FCC
:10060000010ECE6F010ECB6FE552E7CFD9FF12007E
:10061000D9CFE6FFE1CFD9FF000E0001E76ECE197A
:10062000E8AE02D0CE3503D0E750D880CE550AE2EE
:10063000CE5102E0960ECA6F809A8490BA6A828286
:10064000CE6B14D0808A8490FE0EDB40E8403F0BD6
:10065000BB6EFE0EDB50030B100DF3500C09BA6E8F
:10066000FF0ECE5D02E0960ECA6FCE69010ECB6F13
:10067000E552E7CFD9FF1200D9CFE6FFE1CFD9FF8E
:10068000A66AFE0EDB50A96EA680A198A85000D0E5
:10069000E552E7CFD9FF1200D9CFE6FFE1CFD9FF6E
:1006A000FE0EDB50A96EFD0EDB50A86EA66AF29E10
:1006B000A684550EA76EAA0EA76EA682A6B2FED776
:1006C000A694F28EE552E7CFD9FF1200D9CFE6FF0C
:1006D000E1CFD9FF0F0EE1260F0EC16E806A1F0E0B
:1006E000926EFB0E936ED80E946EFC0E956E020EFB
:1006F000966E8194809A8490828283928380400E49
:10070000C76E080EC66E090EC86E280EC66ED18062
:1007100000010F0EC36F0001C35111E00001B66B61
:10072000800EB76F0001B651B71106E0040000015A
:10073000B607000EB75BF6D70001C307ECD7E66A31
:100740009BDFE5520001B66FB76BB6C015F0146AB7
:1007500014C0E6FF15C0E6FF010EE66E8DDFE55220
:10076000E552E7CF15F0E552E7CF14F00001141081
:10077000B66F15C0B7F00A0EDB6AAA0E0001B619F3
:1007800002E1550EB71906E0010EF36E0A0EF3CF23
:10079000DBFF38D01A0EE66E800EE66E000EE66EB7
:1007A000000EE66EE66A91DEF56E050EE15EF5502E
:1007B000AA0E0001981902E1550E991923E0010EC5
:1007C000F36E0A0EF3CFDBFF00010F0EC36F0001C3
:1007D000C35118E00001B66B800EB76F0001B6512F
:1007E000B7110DE004000001B751080B02E083903F
:1007F00001D083800001B607000EB75BEFD7000180
:10080000C307E5D70001C36B320E0001C35D45E2AB
:100810000400C3C0E6FF0001C351156A000F146E47
:10082000030E152214C0E6FF15C0E6FF13DEE552E5
:10083000E552E5520001C351156A000F146E030E14
:10084000152214C0E6FF15C0E6FFB8DDE552E552FB
:100850000001C35D1FE083800001B66B200EB76FFF
:100860000001B651B71106E004000001B607000E02
:10087000B75BF6D783900001B66B200EB76F00010F
:10088000B651B71106E004000001B607000EB75BD1
:10089000F6D7E1D70001C32BB7D70001C36B200EF9
:1008A0000001C35D35E20400C3C0E6FF800E000115
:1008B000C325E66EF1DEE552E552800E0001C32548
:1008C000E66EDADEE5520001C35D1FE083800001C1
:1008D000B66B200EB76F0001B651B71106E00400E9
:1008E0000001B607000EB75BF6D783900001B66B28
:1008F000100EB76F0001B651B71106E004000001F9
:10090000B607000EB75BF6D7E1D70001C32BC7D7F8
:10091000E66A200EE66EE66A9DDDE552E552E55296
:10092000010EE66E210EE66EE66A94DDE552E552B2
:10093000E552050EE66E220EE66EE66A8BDDE552A6
:10094000E552E552020EE66E230EE66EE66A82DDA1
:10095000E552E552E5520A0EDB5034E00001976B98
:100960001E0E0001806F816B00019A6B9B6B9C6B6C
:100970009D6B00019E6B9F6BA06BA16B00010F0E26
:10098000A46F270EA56F0001A26BA36B0001700E70
:10099000A66F010EA76F010E0001A86FA96B050ECF
:1009A0000001AA6FAB6B0400120EE66E9A0EE66EA3
:1009B000000EE66E240EE66EE66AB4DDF56E050EF8
:1009C000E15EF550120EE66E9A0EE66E000EE66ED1
:1009D000240EE66EE66A79DDF56E050EE15EF550F1
:1009E00000019795AA0E0001801902E1550E8119A8
:1009F00007E00001FF0ED88080557F0E815512E27E
:100A0000C80E0001806F816B020EE66E800EE66EEE
:100A1000000EE66E000EE66EE66A84DDF56E050EEB
:100A2000E15EF550AF6AAC6A900EAB6E9D8AF28CB7
:100A30000001D96BD9C0D8F0D9C0D7F0FE0ECF6E67
:100A40000C0ECE6E9D80010ECD6E300E8114000115
:100A5000C86F0001B8690001C56B0001C66BF28E5A
:100A6000310ECB6EBE6ABB6ABD6ABA6ACA84000127
:100A7000CE5103E00001960ECA6F809A8490BA6A44
:100A800082820001CE6BBD6A82940001CD5102E1E9
:100A90000400FBD70001CD6B00013C0E8A6F220ED3
:100AA0008B6F5D0E8C6F7C0E8D6F070E000197159E
:100AB000020A01E106D1030A01E1F3D0010A01E0D3
:100AC0000FD10001010EC66F0001010EC56F0001BC
:100AD000C36BF00E0001C35D01E3E2D0040E000120
:100AE000C55D01E0C8D00400C450146E14C015F0F8
:100AF000146AC35000011424AC6F000E1520AD6FB2
:100B00000001AE6BAF6BADAF02D0AE69AF69000153
:100B1000AF51000AE8AE02D0D8900CD09E0E000172
:100B2000AC5D000E0001AD59000E0001AE59000E83
:100B30000001AF5916E20001C32B0001C351E84088
:100B4000E8403F0BBE6E030E0001C315100DF350BD
:100B50000C09BD6E0001050EC56F0001500EC76F78
:100B60008AD00001010E976FCD0E186ECC0E196E53
:100B70000C0E1A6E800E1B6EC3C007F072EC10F0E4
:100B800005C01CF006C01DF007C01EF008C01FF015
:100B90001CC00AF01DC00BF01EC00CF01FC00DF0F1
:100BA00018C005F019C006F01AC007F01BC008F005
:100BB00019EC17F005C014F006C015F007C016F0C8
:100BC00008C017F0ACC004F0ADC005F0AEC006F030
:100BD000AFC007F05AEC11F005C020F006C021F0BC
:100BE00007C022F008C023F020C00AF021C00BF09B
:100BF00022C00CF023C00DF014C005F015C006F0A3
:100C000016C007F017C008F092EC14F005C08AF087
:100C100006C08BF007C08CF008C08DF000013C0EC0
:100C20008A6F220E8B6F5D0E8C6F7C0E8D6FBD6A8E
:100C30008294040EDB6A050EDB6A060EDB6A070E81
:100C4000DB6A0001966B0001826B836B846B856BA2
:100C50000001866B876B886B896B0001E26B00017A
:100C6000E36B0001AC6BAD6BAE6BAF6B0001C66BA1
:100C70000001C56B15D0050E0001C55D06E1000140
:100C8000C75103E10001010EC56F0001CD5107E01E
:100C90000001CD6B83A002D0839001D0838019D74F
:100CA00020D0040EDB6A050EDB6A060EDB6A070E37
:100CB000DB6A0001966B0001826B836B846B856B32
:100CC00010D083908382040E82C0DBFF050E83C0A8
:100CD000DBFF060E84C0DBFF070E85C0DBFF01D003
:100CE00000D00001B46BB56B0001C66B0001010EB2
:100CF000C56F1A0EE66E800EE66E000EE66E000EF2
:100D0000E66EE66A0FDCF56E050EE15EF550550EF7
:100D1000E66EE66AC1DCE552E552AA0EE66E010E09
:100D2000E66EBADCE552E552080EDB6A090EDB6AB4
:100D30000400080E0001D75D01E09DD00001D96BD1
:100D40000001CF51FF0A37E0010A24E0030A0AE05C
:100D5000EA0A01E085D0E668E6689EDCE552E552E5
:100D6000FF007ED00001FD0EDA6FD1C0D9F0000186
:100D7000D951D92BE66EDB0EE66E000EE66E000151
:100D8000D051E66EE66A65EC02F0F56E050EE15EA6
:100D9000F55066D00001FE0EDA6F0001D051E66E0C
:100DA000E66ADEEC01F0E552E5520001DB6F00017E
:100DB000020ED96F55D0D1C0E6FF0001D051E66ECA
:100DC000E66A2AEC02F0E552E552E5520001DA69E2
:100DD0000001D051E66EE66ADEEC01F0E552E55224
:100DE0000001DB6F0001020ED96F0001D051146EBB
:100DF000156A1A0E145C000E155812E20001D0514B
:100E00000001E46FE56B800E0001E427000E000195
:100E1000E523E4C0E9FFE5C0EAFFD1C0EFFF1FD042
:100E20000001D05123081BE20001D051146E156A55
:100E3000360E145C000E155812E2240E0001D05D2F
:100E40000001E46FE56B9A0E0001E427000E00013B
:100E5000E523E4C0E9FFE5C0EAFFD1C0EFFF00D021
:100E60000001D95108E00001D76B0001010ED86FD5
:100E7000AC8ADAC0ADFF040E0001C55D01E0F7D019
:100E80000001C6516FE1C450146E14C015F0146A0D
:100E9000FE0EC31400011424B96F000E1520BA6FA2
:100EA0000001380ED880B955030EBA5505E200018D
:100EB000380EB96F030EBA6F0001B83513E3B9C02D
:100EC000BBF0BAC0BCF0B9C0BDF0BAC0BEF0B9C08A
:100ED000BFF0BAC0C0F0B9C0C1F0BAC0C2F00001E2
:100EE000B86B3CD00001B851B82BE96EEA6AE9BE94
:100EF000EA68D890E936EA36BB0EE926000EEA2207
:100F0000B9C0EEFFBAC0EDFF00010001BB51000106
:100F1000BD25166E00010001BC510001BE21176EF7
:100F200016500001BF25146E17500001C021156E28
:100F300014500001C1250001B96F15500001C221F4
:100F40000001BA6F020E0F0B000105E0D890BA3312
:100F5000B933E806FBE1030E0001B8170001020EE9
:100F6000C66F82D0020E0001C65D33E1C450146E1C
:100F700014C015F0146AC35000011424B66F000E9B
:100F80001520B76F0001B6510001A25D0001B751F5
:100F90000001A35904E2B6C0A2F0B7C0A3F000015B
:100FA000A4510001B65D0001A5510001B75904E24A
:100FB000B6C0A4F0B7C0A5F00001220EB65D010EC8
:100FC000B75902E2828001D082900001060EC66FFE
:100FD0004BD00001CA5103E00001CA0743D0000111
:100FE000640EA65D000EA75904E2640E0001A66F10
:100FF000A76BC450146E14C015F0146AC3500001DE
:101000001424B66F000E1520B76F0001B651000111
:10101000A65D0001B7510001A75924E2000197B570
:1010200021D0000197850001CE5103E00001960E0A
:10103000CA6F809A8490BA6A82820001CE6B8392D2
:101040008380BD6A82941A0EE66E800EE66E000EF4
:10105000E66E000EE66EE66A92EC02F0F56E050EA4
:10106000E15EF5500001C66B0001010EC56F000185
:10107000CD5102E14BEF0CF0040EE66EA20EE66ECF
:10108000000EE66E2C0EE66EE66A92EC02F0F56E4D
:10109000050EE15EF5500001CE5115E000019E2BDA
:1010A000000E9F23A023A123040EE66E9E0EE66E83
:1010B000000EE66E280EE66EE66A92EC02F0F56E21
:1010C000050EE15EF550070E0001971505E183A0BE
:1010D00002D0839001D08380070E0001971501088C
:1010E00001E0A6D00001CE5156E082C014F083C0CA
:1010F00015F084C016F085C017F0020ED890173294
:10110000163215321432E806F9E1040EDBCF18F07E
:10111000050EDBCF19F0060EDBCF1AF0070EDBCF82
:101120001BF0020ED8901B321A3219321832E80620
:10113000F9E11450181809E11550191806E1165074
:101140001A1803E117501B1800E125E10001CA51EC
:1011500022E1000197850001CE5103E00001960EC7
:10116000CA6F809A8490BA6A82820001CE6B8392A1
:101170008380BD6A82941A0EE66E800EE66E000EC3
:10118000E66E000EE66EE66A92EC02F0F56E050E73
:10119000E15EF5504DD0F29E0B0E82C0DBFF0C0ECF
:1011A00083C0DBFF0D0E84C0DBFF0E0E85C0DBFFAE
:1011B000F28E0001CB5135E00001CB6B040EE66EE0
:1011C000D9500B0FE66E000EDA20E66E020EE66EC8
:1011D000E66A92EC02F0F56E050EE15EF550040E43
:1011E000E66ED9500B0FE66E000EDA20E66EE66A68
:1011F000010EE66E92EC02F0F56E050EE15EF55022
:10120000040EE66ED9500B0FE66E000EDA20E66E85
:10121000E66A020EE66E92EC02F0F56E050EE15EF5
:10122000F55083A003D08390838202D08392838081
:101230000001B451B51120E00001B407000EB55B08
:10124000FF0E0001B415146E7F0E0001B515156E6A
:101250001450151011E10001B451B51104E0000162
:10126000B46BB56B09D00001AA510001B46F800EB8
:101270000001AB110001B56F070E000197150208C0
:1012800001E007D30001CE5156E082C014F083C0C4
:1012900015F084C016F085C017F0020ED8901732F2
:1012A000163215321432E806F9E1040EDBCF18F0DD
:1012B000050EDBCF19F0060EDBCF1AF0070EDBCFE1
:1012C0001BF0020ED8901B321A3219321832E8067F
:1012D000F9E11450181809E11550191806E11650D3
:1012E0001A1803E117501B1800E125E10001CA514B
:1012F00022E1000197850001CE5103E00001960E26
:10130000CA6F809A8490BA6A82820001CE6B8392FF
:101310008380BD6A82941A0EE66E800EE66E000E21
:10132000E66E000EE66EE66A92EC02F0F56E050ED1
:10133000E15EF550AED2F29E040E82C0DBFF050ED8
:1013400083C0DBFF060E84C0DBFF070E85C0DBFF1A
:10135000F28E0001CB5135E00001CB6B040EE66E3E
:10136000D950040FE66E000EDA20E66E020EE66E2D
:10137000E66A92EC02F0F56E050EE15EF550040EA1
:10138000E66ED950040FE66E000EDA20E66EE66ACD
:10139000010EE66E92EC02F0F56E050EE15EF55080
:1013A000040EE66ED950040FE66E000EDA20E66EEB
:1013B000E66A020EE66E92EC02F0F56E050EE15E54
:1013C000F550040EDBCF20F0050EDBCF21F0060E2A
:1013D000DBCF22F0070EDBCF23F020C004F021C0CA
:1013E00005F022C006F023C007F05AEC11F005C04A
:1013F0001CF006C01DF007C01EF008C01FF092C010
:101400000AF093C00BF094C00CF095C00DF01CC016
:1014100005F01DC006F01EC007F01FC008F09CECD0
:1014200012F005C018F006C019F007C01AF008C085
:101430001BF08EC00AF08FC00BF090C00CF091C072
:101440000DF018C005F019C006F01AC007F01BC057
:1014500008F092EC14F005C014F006C015F007C0B7
:1014600016F008C017F014C00AF015C00BF016C033
:101470000CF017C00DF08AC005F08BC006F08CC0D0
:1014800007F08DC008F019EC17F09DEC17F006C0BE
:10149000B0F007C0B1F0B0C014F0B1C015F0D890F2
:1014A00015321432D890153214321450BE6E030E19
:1014B0000001B015146E156A040ED8901436153656
:1014C000E804FBE10C0E1410BD6E0001960ED880EE
:1014D000B955000EBA5548E2B9C006F0BAC007F0D7
:1014E000A7EC10F005C018F006C019F007C01AF0FC
:1014F00008C01BF08EC00AF08FC00BF090C00CF03B
:1015000091C00DF018C005F019C006F01AC007F020
:101510001BC008F019EC17F005C014F006C015F058
:1015200007C016F008C017F092C00AF093C00BF085
:1015300094C00CF095C00DF014C005F015C006F075
:1015400016C007F017C008F09DEC12F03BEC18F045
:1015500004C0ACF005C0ADF006C0AEF007C0AFF0FF
:101560000001B96BBA6B8FD0300E00019715200ABD
:1015700040E0200A01E07BD0186A196A240E1A6E36
:10158000860E1B6E8EC00AF08FC00BF090C00CF060
:1015900091C00DF018C005F019C006F01AC007F090
:1015A0001BC008F019EC17F005C014F006C015F0C8
:1015B00007C016F008C017F092C00AF093C00BF0F5
:1015C00094C00CF095C00DF014C005F015C006F0E5
:1015D00016C007F017C008F09DEC12F03BEC18F0B5
:1015E00004C0ACF005C0ADF006C0AEF007C0AFF06F
:1015F0004AD0186A800E196E4C0E1A6E880E1B6E39
:101600008EC00AF08FC00BF090C00CF091C00DF0AE
:1016100018C005F019C006F01AC007F01BC008F08A
:1016200019EC17F005C014F006C015F007C016F04D
:1016300008C017F092C00AF093C00BF094C00CF0F1
:1016400095C00DF014C005F015C006F016C007F0E7
:1016500017C008F09DEC12F03BEC18F004C0ACF0A1
:1016600005C0ADF006C0AEF007C0AFF00CD0040E60
:10167000DBCFACF0050EDBCFADF0060EDBCFAEF06E
:10168000070EDBCFAFF0D950040FE96EDACFEAFFD7
:10169000EE500001AC5D186EEE500001AD59196EB0
:1016A000EE500001AE591A6EEE500001AF591B6E9C
:1016B0000001800E1B151EE0D950040FE96EDACF31
:1016C000EAFFEE500001AC5D146EEE500001AD5922
:1016D000156EEE500001AE59166EEE500001AF5976
:1016E000176E000E146C151E1522161E1622171EDC
:1016F000172215D0D950040FE96EDACFEAFFEE5069
:101700000001AC5D146EEE500001AD59156EEE5047
:101710000001AE59166EEE500001AF59176E80C031
:101720001CF081C01DF01E6A1F6A1F501718E8AE1A
:1017300002D0173408D014501C5C15501D58165098
:101740001E5817501F5801E398D00001B551800B67
:1017500001E086D00001CE511DE100019A2B000E60
:101760009B239C239D23040EE66E9A0EE66E000ECC
:10177000E66E240EE66EE66A92EC02F0F56E050E59
:10178000E15EF5500001B451B51104E1A8C0B4F018
:10179000A9C0B5F0040EDBCF05F0050EDBCF06F0D7
:1017A000060EDBCF07F0070EDBCF08F00850000174
:1017B000AF19E8AE02D0AF350CD00001AC51055CDA
:1017C0000001AD5106580001AE5107580001AF515C
:1017D000085817E2000E0001E76E9619E8AE02D035
:1017E000963503D0E750D880965506E2C80EE66ECF
:1017F000DDEC02F0E55205D0C80EE66E08EC03F011
:10180000E552040EDBCF05F0050EDBCF06F0060E29
:10181000DBCF07F0070EDBCF08F00001AF5108184F
:10182000E8AE02D008340CD005500001AC5D065083
:101830000001AD5907500001AE5908500001AF59E1
:101840000EE20001963506E3C80EE66EDDEC02F00E
:10185000E55205D0C80EE66E08EC03F0E5520CD058
:101860000001CE5103E00001960ECA6F809A849069
:10187000BA6A82820001CE6B0CD00001CE5103E027
:101880000001960ECA6F809A8490BA6A8282000123
:10189000CE6B0001CD6B070E00019715020A01E126
:1018A00028D3030A01E0E3D3080E0001D75D01E06D
:1018B000F2D2F00E0001CF5D01E3EDD2170E000170
:1018C000CF5D01E1E8D20001D76B0001010ED96FB5
:1018D0000001CF51050A01E16AD2010A01E1E9D113
:1018E000070A01E1B1D1010A01E189D1030A01E04E
:1018F000D0D20001D05104E0AC8A010EAD6E7ED191
:101900000001CE5103E00001960ECA6F809A8490C8
:10191000BA6A82820001CE6BC00E0001971527E1E2
:101920001A0EE66E800EE66E000EE66E000EE66E95
:10193000E66A65EC02F0F56E050EE15EF550070E05
:1019400000019715020813E1C00E00019713839060
:1019500083820001B46BB56B0001CB6B0001C66BD9
:101960000001010EC56FAC8A010EAD6E94D2C00E9F
:1019700000019715C00801E03FD10001965101E137
:101980003BD10001D139F00B02090001976F000132
:10199000AA0E986F550E996F86C004F087C005F0A7
:1019A00088C006F089C007F05AEC11F005C014F0A9
:1019B00006C015F007C016F008C017F00A0E1C6E1E
:1019C000D70E1D6E230E1E6E840E1F6E0001E25197
:1019D0000001E35D246E24C007F072EC10F005C036
:1019E00020F006C021F007C022F008C023F020C07C
:1019F0000AF021C00BF022C00CF023C00DF01CC077
:101A000005F01DC006F01EC007F01FC008F019EC5D
:101A100017F005C018F006C019F007C01AF008C08A
:101A20001BF018C00AF019C00BF01AC00CF01BC054
:101A30000DF014C005F015C006F016C007F017C071
:101A400008F092EC14F005C08EF006C08FF007C0CD
:101A500090F008C091F00A0E1C6ED70E1D6E230E7A
:101A60001E6E840E1F6EE2C007F072EC10F005C00F
:101A700020F006C021F007C022F008C023F020C0EB
:101A80000AF021C00BF022C00CF023C00DF01CC0E6
:101A900005F01DC006F01EC007F01FC008F019ECCD
:101AA00017F005C018F006C019F007C01AF008C0FA
:101AB0001BF08EC00AF08FC00BF090C00CF091C0EC
:101AC0000DF018C005F019C006F01AC007F01BC0D1
:101AD00008F019EC17F005C014F006C015F007C0A7
:101AE00016F008C017F00A6A0B6A800E0C6E7F0EA3
:101AF0000D6E14C005F015C006F016C007F017C033
:101B000008F019EC17F005C092F006C093F007C07A
:101B100094F008C095F0F29E040E82C0DBFF050E23
:101B200083C0DBFF060E84C0DBFF070E85C0DBFF32
:101B3000F28E8390838204001A0EE66E800EE66EAB
:101B4000000EE66E000EE66EE66A92EC02F0F56EAE
:101B5000050EE15EF550040EE66ED950040FE66EF8
:101B6000000EDA20E66EE66A010EE66E92EC02F0F6
:101B7000F56E050EE15EF550040EE66ED950040FC9
:101B8000E66E000EDA20E66EE66A020EE66E92EC73
:101B900002F0F56E050EE15EF5500400F29EA96AB2
:101BA000550EA86EA66AA684550EA76EAA0EA76E3D
:101BB000A682A6B2FED70400A198010EA96EAA0EB5
:101BC000A86EA66AA684550EA76EAA0EA76EA68258
:101BD000A6B2FED70400A198A694F28E0001B46BC1
:101BE000B56B0001CB6B0001C66B0001010EC56F28
:101BF000AC8A010EAD6E02D0AC8AAD6A4CD1C00E7B
:101C0000000197150FE11A0EE66E800EE66E000ECB
:101C1000E66E000EE66EE66A92EC02F0F56E050ED8
:101C2000E15EF550AC8A020EAD6E0001978DF29E1A
:101C300082C086F083C087F084C088F085C089F0B8
:101C4000F28ED0C0E3F027D1C00E000197150FE14E
:101C50001A0EE66E800EE66E000EE66E000EE66E62
:101C6000E66A92EC02F0F56E050EE15EF550AC8A84
:101C7000030EAD6E0001978FF29E000197AD10D05C
:101C8000000182510001865F000183510001875BE2
:101C9000000184510001885B000185510001895BCE
:101CA0000001826B836B846B856BF28ED0C0E2F097
:101CB000F2D0080ED0C0DBFFF29E080EDB5010E021
:101CC000000196510CE1040E82C0DBFF050E83C0BB
:101CD000DBFF060E84C0DBFF070E85C0DBFF62D092
:101CE000000196515FE1090EDBCF14F0000EE76EA4
:101CF0001418E8AE02D0143403D0E750D88014543E
:101D000026E2040EDBCF05F0050EDBCF06F0060E53
:101D1000DBCF07F0070EDBCF08F008500001851974
:101D2000E8AE02D085350CD000018251055C00017F
:101D30008351065800018451075800018551085805
:101D400004E20001010E966F02D000019669090EAF
:101D5000DBCF14F0143426E3040EDBCF05F0050EC0
:101D6000DBCF06F0060EDBCF07F0070EDBCF08F067
:101D7000000185510818E8AE02D008340CD0055097
:101D80000001825D0650000183590750000184590B
:101D900008500001855904E20001010E966F02D03F
:101DA00000019669F28EAC8A040EAD6E74D0C00E3E
:101DB0000001971300019669D0C014F014C015F00B
:101DC000146A0001D15100011410826F15C083F014
:101DD0000001846B856B83AF02D084698569000E36
:101DE0000001826D0001831F83230001841F84236F
:101DF0000001851F8523020E0001D89082378337AA
:101E000084378537E806F9E1D2C014F014C015F024
:101E1000146A0001D35100011410866F15C087F0B9
:101E20000001886B896B87AF02D08869896986C099
:101E300014F087C015F088C016F089C017F0020EA4
:101E4000D8901436153616361736E806F9E1820EA4
:101E5000E96E000EEA6E1450EE5C0001866F1550BC
:101E6000EE580001876F1650EE580001886F17502A
:101E7000EE580001896FD4C0E2F0D5C0E3F0000154
:101E8000040EE26F0001140EE36FAC8A050EAD6E16
:101E900002D00001D96B080EDB501EE00001B551E5
:101EA000800B1AE10001B451B51104E1A8C0B4F0EF
:101EB000A9C0B5F0080EDB0406E1C80EE66EDDEC45
:101EC00002F0E55205D0C80EE66E08EC03F0E552CC
:101ED000090ECEC0DBFF0CD00001CE5103E00001A3
:101EE000960ECA6F809A8490BA6A82820001CE6B85
:101EF000F1D0080E0001D75D3EE1F00E0001CF5D8C
:101F00003AE2170E0001CF5D36E00001D76B000109
:101F1000CF0531E10001D0512EE00001CE5103E0A8
:101F20000001960ECA6F809A8490BA6A828200017C
:101F3000CE6B83800001010E976F080EDB6A090EDD
:101F4000DB6A0001966B040EDB6A050EDB6A060E87
:101F5000DB6A070EDB6A0001866B876B886B896B17
:101F60000001E26B0001E36B0001010ED96FAC8A46
:101F7000010EAD6EAFD00001CE5101E177D0F29EDF
:101F800082C0DFFF010E83C0DBFF020E84C0DBFFD7
:101F9000030E85C0DBFFF28ED9CFE9FFDACFEAFF6F
:101FA000EE500001AC5D186EEE500001AD59196E97
:101FB000EE500001AE591A6EEE500001AF591B6E83
:101FC0000001800E1B151DE0D9CFE9FFDACFEAFF33
:101FD000EE500001AC5D146EEE500001AD59156E6F
:101FE000EE500001AE59166EEE500001AF59176E5B
:101FF000000E146C151E1522161E1622171E17220F
:1020000014D0D9CFE9FFDACFEAFFEE500001AC5D82
:10201000146EEE500001AD59156EEE500001AE5930
:10202000166EEE500001AF59176E1750000AE8AE59
:1020300002D0D89008D0320E145C000E1558000E55
:102040001658000E175812E20001010ECB6F000166
:10205000B46BB56B0001CE5103E00001960ECA6F60
:10206000809A8490BA6A82820001CE6B33D0080EC7
:102070000001D75D2EE1F00E0001CF5D2AE2170EC0
:102080000001CF5D26E00001CF0521E10001010E36
:10209000D96FAC8A0001D05119E0010EAD6E00017C
:1020A000010E976F0001966B0001826B836B846B4E
:1020B000856B040EDB6A050EDB6A060EDB6A070E13
:1020C000DB6A080EDB6A090EDB6A01D0AD6A00012B
:1020D000D76B00D098EF06F0D9CFE1FFE552E7CFFC
:0420E000D9FF120012
:0C20E400860E086E0E6A066A056A046A21
:1020F00086EF10F0860E086E07C00EF0066A056ABD
:10210000046AE86A07AE86EF10F0076C136AE86AA3
:1021100007644CEF11F0F00E0714E86692EF10F030
:10212000073A1384D89007BEA2EF10F00736132A9F
:1021300007BEA2EF10F00736132A07BEA2EF10F079
:102140000736132A1350085E0EAE079E000C8E0E43
:10215000086E0E6A056A046ABBEF10F08E0E086EF8
:1021600007C00EF0056A046A07AEBBEF10F0066CFC
:10217000071EE86A0722136AE86A0764E4EF10F0B2
:10218000F00E0714E866CDEF10F0073A06380F0B93
:1021900007260638F00B066E1384D89007BEE0EFD2
:1021A00010F006360736132A07BEE0EF10F00636A9
:1021B0000736132A07BEE0EF10F006360736132A5B
:1021C0001350085E52EF11F006C007F0066AE86A85
:1021D000138607644CEF11F0F00E0714E866F3EF76
:1021E00010F0073A1384D89007BEE0EF10F00736DE
:1021F000132A07BEE0EF10F00736132A07BEE0EF00
:1022000010F00736132AE0EF10F00F800FAEFF0C2E
:10221000076A0EAE076807C006F007C005F007C0E2
:1022200004F00E360732FF0C0F800FAEFF0C076A6A
:102230000EAE076807C006F007C005F00E3607327D
:10224000FF0C0F800FAEFF0C076A0EAE076807C0C9
:1022500006F00E360732FF0C0F800FAEFF0C076A38
:102260000EAE07680E360732FF0C0F820FAEFF0C62
:1022700008680768066805680E360732FF0C0F8489
:102280000FAEFF0C010E086E076A066A056A0E366D
:102290000732FF0C0F86FF0C076A066A056A046A9C
:1022A000086A000C0EAE079E000C9E0E086E0E6AA9
:1022B00069EF11F09E0E086E07C00EF007AE69EFD1
:1022C00011F0E86A046C051E061E071E0522062290
:1022D00007220750FF0BD8B4CEEF11F0F00BD8B4A3
:1022E000A7EF11F0E86A07BE90EF11F0D89004361E
:1022F000053606360736E82A07BE8CEF11F004369D
:10230000053606360736E82A07BE8CEF11F004368C
:10231000053606360736E82A08643FEF11F0085EF6
:102320000FBC04AE52EF11F0D880800E046405306B
:10233000E86A052206220722D8A052EF11F00732E0
:1023400006320532084A35EF11F052EF11F005C0A0
:102350000AF007C00CF0D8900734190FF66E250E5E
:10236000F76AF722000EF86AF8220A00F550040214
:10237000F3CF04F0F4CF05F00602F3CF06F0F4CF6C
:1023800007F00A02F3500526F4500626F5500C0219
:10239000F35007260800F5508CEF11F00650076E39
:1023A000FF0BD8B417EF12F005C006F004C005F01B
:1023B000046A0750F00BD8B4F7EF11F0080E07BE0F
:1023C0008CEF11F0D890053606360736E82A07BE9E
:1023D0008CEF11F0053606360736E82A07BE8CEF7B
:1023E00011F0053606360736E82A8CEF11F006C0E4
:1023F0000BF0D8900734190FF66E250EF76AF72206
:10240000000EF86AF8220A00F5500502F3CF05F035
:10241000F4CF06F00702F3CF07F00B02F3500626C5
:10242000F45007260800F550080F8CEF11F0055006
:10243000076EFF0BD8B457EF12F004C006F0056A20
:10244000046A0750F00BD8B43CEF12F0100E07BE30
:102450008CEF11F0D89006360736E82A07BE8CEFCD
:1024600011F006360736E82A07BE8CEF11F0063663
:102470000736E82A8CEF11F007C00CF0D89007342B
:10248000190FF66E250EF76AF722000EF86AF82289
:102490000A00F5500602F3CF06F0F4CF07F00C0265
:1024A000F35007260800F550100F8CEF11F0045080
:1024B000076EFF0BD8B44CEF11F0066A056A046A88
:1024C0000750F00BD8B478EF12F0180E07BE8CEF5F
:1024D00011F0D8900736E82A07BE8CEF11F00736C6
:1024E000E82A07BE8CEF11F00736E82A8CEF11F0CE
:1024F000D8900734190FF66E250EF76AF722000EF2
:10250000F86AF8220A00F5500702F3CF07F0080036
:10251000F550180F8CEF11F00000078006400640C0
:1025200005200520052005200410041004100410C7
:1025300004100410041004100C7E07500C18136EC5
:10254000046A08500D648CEF13F00CC00EF00C8E72
:10255000078E08C012F00DC008F0E86A1264DEEFC2
:1025600012F012500D5ED8B47EEF13F0070E0D641A
:102570004CEF13F00D5E05C004F006C005F007C077
:1025800006F0076A0D4E7EEF13F00D6421EF13F095
:102590000D5E05C004F006C005F0066A0D4E7EEF24
:1025A00013F00D64FFEF12F00D5E05C004F0056A34
:1025B0000D4E7EEF13F00D64E6EF12F00EC007F043
:1025C0000BC006F00AC005F0046A000C030E0D648F
:1025D000F1EF12F00D5E04380F0B046E0D4E7EEF1E
:1025E00013F0D89004320D4E7EEF13F0D8900432E1
:1025F0000D4E7EEF13F0D89004327EEF13F0030EF1
:102600000D6410EF13F00D5E04380F0B046E0538E7
:10261000F00B042605380F0B056E0D4E7EEF13F000
:10262000D890053204320D4E7EEF13F0D89005326B
:1026300004320D4E7EEF13F0D890053204327EEF57
:1026400013F0030E0D6438EF13F00D5E04380F0B1A
:10265000046E0538F00B042605380F0B056E06389E
:10266000F00B052606380F0B066E0D4E7EEF13F0AD
:10267000D8900632053204320D4E7EEF13F0D8901A
:102680000632053204320D4E7EEF13F0D89006323A
:10269000053204327EEF13F0030E0D6469EF13F080
:1026A0000D5E04380F0B046E0538F00B0426053858
:1026B0000F0B056E0638F00B052606380F0B066E5D
:1026C0000738F00B062607380F0B076E0D4E7EEF0E
:1026D00013F0D89007320632053204320D4E7EEFE9
:1026E00013F0D89007320632053204320D4E7EEFD9
:1026F00013F0D8900732063205320432096A13AE5D
:102700006DEF14F0046C051E061E071EE86A052214
:10271000062207226DEF14F00D6690EF13F0000C07
:10272000096A07C00EF0078E0C8E0D50085C0D6E06
:10273000D8B461EF14F0070E0D642FEF14F00D5EA6
:102740000AC009F00BC00AF00CC00BF00C6A0D4E69
:1027500061EF14F0070E0D6404EF14F00D5E0AC073
:1027600009F00BC00AF00B6A0D4E61EF14F0070E72
:102770000D64E2EF13F00D5E0AC009F00A6A0D4E17
:1027800061EF14F0070E0D64C9EF13F00EC007F0EF
:10279000000C030E0D64D4EF13F00D5E09380F0B1F
:1027A000096E0D4E61EF14F0D89009320D4E61EFB5
:1027B00014F0D89009320D4E61EF14F0D890093220
:1027C00061EF14F0030E0D64F3EF13F00D5E0938A2
:1027D0000F0B096E0A38F00B09260A380F0B0A6E28
:1027E0000D4E61EF14F0D8900A3209320D4E61EFB0
:1027F00014F0D8900A3209320D4E61EF14F0D890DF
:102800000A32093261EF14F0030E0D641BEF14F06D
:102810000D5E09380F0B096E0A38F00B09260A38CD
:102820000F0B0A6E0B38F00B0A260B380F0B0B6ED2
:102830000D4E61EF14F0D8900B320A3209320D4E72
:1028400061EF14F0D8900B320A3209320D4E61EF6D
:1028500014F0D8900B320A32093261EF14F0030EF3
:102860000D644CEF14F00D5E09380F0B096E0A3839
:10287000F00B09260A380F0B0A6E0B38F00B0A26EC
:102880000B380F0B0B6E0C38F00B0B260C380F0BA4
:102890000C6E0D4E61EF14F0D8900C320B320A32F0
:1028A00009320D4E61EF14F0D8900C320B320A321F
:1028B00009320D4E61EF14F0D8900C320B320A320F
:1028C0000932046A13AE6DEF14F0096C0A1E0B1E78
:1028D0000C1EE86A0A220B220C22095004260A5018
:1028E00005220B5006220C50072213BE84EF14F071
:1028F000D8A090EF11F00732063205320432083EBC
:1029000090EF11F035EF11F0D8B069EF11F0E86AEF
:10291000046C051E061E071E0522062207220E7ED7
:1029200069EF11F0106AE86A0D644AEF11F008646B
:102930004CEF11F007500C180E6E078E0C8E0B34F6
:102940000C341336D890E8361336320FF66E2C0E50
:10295000F76E1350010BF722F86A000EF8220A00F6
:10296000F5CF02F00A00F5CF13F00800F5CF12F012
:102970000250125C026ED8900A340202F4CFF7FFC4
:102980000B340202F3CFE8FFF726D8B0F42A116A1D
:10299000F750115EF450125AE86A135A07C002F059
:1029A00006C0F7FF05C0F6FF05501102F4CF03F093
:1029B00006501202F4CF05F0F3CF04F01102F350E9
:1029C0000326F4500422E86A0522F6501202F3505E
:1029D0000326F4500422E86A052207501102F3503E
:1029E0000426F450052207501202066AE86A0622FD
:1029F000F3500526F4500622F6501302F350042635
:102A0000F4500522076AE86A06220722F7501302EB
:102A1000F3500526F4500622E86A072202501302FA
:102A2000F3500626F450072207BE1CEF15F00436BB
:102A300005360636073610060CC002F00BC0F7FF4D
:102A40000AC0F6FF0A501102F4CF03F00B50120235
:102A5000F4CF0AF0F3CF09F01102F3500326F4503B
:102A60000922E86A0A22F6501202F3500326F450B3
:102A70000922E86A0A220C501102F3500926F45088
:102A80000A220C5012020B6AE86A0B22F3500A2643
:102A9000F4500B22F6501302F3500926F4500A2288
:102AA0000C6AE86A0B220C22F7501302F3500A2634
:102AB000F4500B22E86A0C2202501302F3500B264A
:102AC000F4500C220CAE0CBC6CEF15F0033609363A
:102AD0000A360B360C36102A096C0A1E0B1E0C1E09
:102AE000E86A0A220B220C2207C013F006C012F07B
:102AF00005C011F004C0F6FF05500A02F4CF03F040
:102B000006500902F450032606500A02046AE86AD5
:102B10000422F3500326F4500422F6500B02F45022
:102B20000326056AE86A0422052211500B02F350BD
:102B30000326F4500422E86A052212500B02F350D7
:102B40000426F450052207500A02F3500426F450DC
:102B5000052207500B02066AE86A0622F350052692
:102B6000F450062213500902F3500326F4500422B5
:102B7000E86A0522062213500C02F4CF07F0F35046
:102B80000626E86A0722F6500C02F3500326F4509A
:102B90000422E86A05220622072211500C02F35093
:102BA0000426F4500522E86A0622072212500C027D
:102BB000F3500526F4500622E86A072207BEEEEF1E
:102BC00015F00436053606360736100607BEEEEF5A
:102BD00015F0043605360636073610060D50085E29
:102BE000800ED8A0FBEF15F010240826D8B035EFE2
:102BF00011F000EF16F010240826D8A03FEF11F0D6
:102C00000FBC04AE15EF16F0D880800E04640530BA
:102C1000E86A052206220722D8A015EF16F007322F
:102C200006320532084A35EF11F00EAE079E000C51
:102C3000FFFF01FF04FE09FD10FC19FB23FA30F928
:102C40003EF84EF760F674F58AF4A1F3BAF2D5F1C6
:102C5000F1F00FF02FEF50EE73ED98ECBEEBE5EADC
:102C60000FEA39E966E893E7C3E6F3E526E559E4B8
:102C70008EE3C5E2FCE136E170E0ACDFE9DE28DEA0
:102C800068DDA9DCEBDB2FDB74DABAD902D94AD8CC
:102C900094D7DFD62CD679D5C7D417D468D3BAD277
:102CA0000DD261D1B7D00DD064CFBDCE17CE71CDCE
:102CB000CDCC29CC87CBE6CA46CAA6C908C96AC802
:102CC000CEC733C798C6FEC566C5CEC437C4A1C338
:102CD0000CC378C2E5C152C1C1C030C0A0BF11BF92
:102CE00083BEF6BD69BDDDBC52BCC8BB3FBBB6BA36
:102CF0002FBAA8B921B99CB817B893B710B78DB639
:102D00000BB68AB50AB58AB40BB48DB30FB392B2C1
:102D100016B29BB120B1A6B02CB0B3AF3BAFC3AEDF
:102D20004CAED6AD60ADEBAC77AC03AC8FAB1DABAE
:102D3000ABAA39AAC8A958A9E8A879A80BA89CA742
:102D40002FA7C2A656A6EAA57FA514A5AAA440A4AB
:102D5000D7A36EA306A39FA238A2D1A16BA106A1FF
:102D6000A1A03CA0D89F749F119FAF9E4D9EEB9D4C
:102D70008A9D299DC99C699C0A9CAB9B4C9BEE9AA1
:102D8000919A349AD7997B991F99C49869980E980B
:102D9000B4975A970197A8965096F895A09549959B
:102DA000F2949C944694F0939B934693F1929D9257
:102DB0004992F691A3915091FE90AC905A9009904F
:102DC000B88F688F178FC88E788E298EDA8D8C8D8C
:102DD0003E8DF08CA38C568C098CBC8B708B248B15
:102DE000D98A8E8A438AF889AE8964891B89D288F8
:102DF00089884088F887AF8768872087D986928638
:102E00004C860586BF8579853485EF84AA846584E0
:102E10002184DD83998356831283CF828D824A82F7
:102E20000882C681858143810281C1808180408082
:102E30000180046AE86A0D6208644CEF11F00750E3
:102E40000C180E6E0D5008267E0ED8A02EEF17F02F
:102E5000085ED8B035EF11F032EF17F0085ED8A059
:102E60003FEF11F0078E0C8E07C013F006C012F072
:102E700005C011F005500A02F4CF03F006500B0212
:102E8000F4CF05F0F3CF04F00A02F3500326F45018
:102E90000422E86A052211500B02F3500326F45075
:102EA0000422E86A052207500A02F3500426F4506F
:102EB000052207500B02066AE86A0622F35005262F
:102EC000F450062211500C02F3500426F45005224F
:102ED000076AE86A0622072212500C02F350052600
:102EE000F4500622E86A072213500C02F35006261B
:102EF000F450072207BE85EF17F004360536063674
:102F000007360806D8B43FEF11F00FBC04AE9AEFB5
:102F100017F0D880800E04640530E86A0522062286
:102F20000722D8A09AEF17F0073206320532084A76
:102F300035EF11F00EAE079E000CE86A0864000C35
:102F400007C00EF0078E8E0E085CE8AE21EF11F080
:102F5000E86C086E070E0864FDEF17F0085E06C007
:102F600005F007C006F0076A084E26EF18F0070EB6
:102F70000864DBEF17F0085E06C005F0066A084E2D
:102F800026EF18F0030E0864CDEF17F0085E053841
:102F90000F0B056E084E26EF18F0D8900532084E3C
:102FA00026EF18F0D8900532084E26EF18F0D8908A
:102FB000053226EF18F0030E0864ECEF17F0085EF8
:102FC00005380F0B056E0638F00B052606380F0B7B
:102FD000066E084E26EF18F0D89006320532084EDD
:102FE00026EF18F0D89006320532084E26EF18F07A
:102FF000D8900632053226EF18F0030E086414EF5D
:1030000018F0085E05380F0B056E0638F00B052624
:1030100006380F0B066E0738F00B062607380F0B25
:10302000076E084E26EF18F0D890073206320532A8
:10303000084E26EF18F0D890073206320532084EB7
:1030400026EF18F0D8900732063205320FBC05AED5
:1030500034EF18F0D880800E05640630E86A062246
:10306000072207BE21EF11F00EAE000C066C071E02
:10307000E86A0722000C046AE86A0864000C07C0CA
:103080000EF0078E036A9E0E085CE8AE05EF11F0A5
:10309000E86C086E070E086408EF19F0085E04C0BB
:1030A00003F005C004F006C005F007C006F0076A8B
:1030B000084E3EEF19F00864D9EF18F0085E04C01E
:1030C00003F005C004F006C005F0066A084E3EEFA6
:1030D00019F00864B3EF18F0085E04C003F005C0EF
:1030E00004F0056A084E3EEF19F0086496EF18F0F8
:1030F000085E04C003F0046A084E3EEF19F0030EA8
:10310000086488EF18F003380F0B036E3EEF19F0D8
:10311000D8900332084E3EEF19F0D8900332084E93
:103120003EEF19F0D89003323EEF19F0030E086419
:10313000A2EF18F0085E0438036E0F0B046E084E01
:103140003EEF19F0D89004320332084E3EEF19F0EA
:10315000D89004320332084E3EEF19F0D890043272
:1031600003323EEF19F0030E0864C5EF18F0085E55
:103170000438036E0F0B046E0538F00B0426053877
:103180000F0B056E084E3EEF19F0D8900532043251
:103190000332084E3EEF19F0D89005320432033264
:1031A000084E3EEF19F0D8900532043203323EEF5C
:1031B00019F0030E0864F1EF18F0085E0438036E8E
:1031C0000F0B046E0538F00B042605380F0B056E47
:1031D0000638F00B052606380F0B066E084E3EEF3C
:1031E00019F0D8900632053204320332084E3EEF11
:1031F00019F0D8900632053204320332084E3EEF01
:1032000019F0D89006320532043203323EEF19F03D
:10321000030E086426EF19F0085E0438036E0F0BE6
:10322000046E0538F00B042605380F0B056E0638C2
:10323000F00B052606380F0B066E0738F00B062636
:1032400007380F0B076E084E3EEF19F0D890073283
:103250000632053204320332084E3EEF19F0D890A0
:1032600007320632053204320332084E3EEF19F0BF
:10327000D890073206320532043203320FBC03AE57
:103280004EEF19F0D880800E03640430E86A0422FF
:1032900005220622072207BE05EF11F00EAE000C34
:1032A000046C051E061E071EE86A05220622072278
:0232B000000C10
:0E32B2002A0EF66E020EF76E000EF86E000188
:1032C0000900F550EB6F0900F550EC6F03E1EB6777
:1032D00001D03DD00900F550E66F0900F550E76FC9
:1032E0000900F550E86F09000900F550E96E090082
:1032F000F550EA6E090009000900F550E96F090070
:10330000F550EA6F09000900F6CFEDF0F7CFEEF0C7
:10331000F8CFEFF0E6C0F6FFE7C0F7FFE8C0F8FF30
:103320000001E95302E1EA5307E00900F550EE6EAF
:10333000E907F8E2EA07F9D7EDC0F6FFEEC0F7FFBC
:10334000EFC0F8FF0001EB07000EEC5BBFD71200E7
:1033500015EE00F025EE00F0F86A0F8C59EC19F02C
:0833600066EC03F0FDD712003A
:00000001FF
